 FileCase

 Timestamp is 537255c0 (Tue May 13 21:26:24 2014)

 Preferred load address is 0000000180000000

 Start         Length     Name                   Class
 0001:00000000 00000048H .idata$5                CODE
 0001:00000050 000002d2H .rdata                  CODE
 0001:00000330 00002c83H .text                   CODE
 0001:00002fb8 000002bcH .xdata                  CODE
 0001:00003274 00000014H .idata$2                CODE
 0001:00003288 00000014H .idata$3                CODE
 0001:000032a0 00000048H .idata$4                CODE
 0001:000032e8 00000074H .idata$6                CODE
 0001:00003360 00000091H .edata                  CODE
 0002:00000000 00000000H .data                   DATA
 0002:00000000 000006c0H .bss                    DATA
 0003:00000000 000002b8H .pdata                  DATA
 0004:00000000 00000058H .rsrc$01                DATA
 0004:00000060 00000390H .rsrc$02                DATA

  Address         Publics by Value              Rva+Base               Lib:Object

 0000:00000000       ___safe_se_handler_count   0000000000000000     <absolute>
 0000:00000000       ___safe_se_handler_table   0000000000000000     <absolute>
 0000:00000000       __ImageBase                0000000180000000     <linker-defined>
 0001:00000000       __imp_lstrcpynW            0000000180001000     kernel32:KERNEL32.dll
 0001:00000008       __imp_lstrlenW             0000000180001008     kernel32:KERNEL32.dll
 0001:00000010       __imp_lstrcpyW             0000000180001010     kernel32:KERNEL32.dll
 0001:00000018       __imp_MoveFileW            0000000180001018     kernel32:KERNEL32.dll
 0001:00000020       __imp_lstrcatW             0000000180001020     kernel32:KERNEL32.dll
 0001:00000028       __imp_HeapFree             0000000180001028     kernel32:KERNEL32.dll
 0001:00000030       __imp_GetProcessHeap       0000000180001030     kernel32:KERNEL32.dll
 0001:00000038       __imp_HeapAlloc            0000000180001038     kernel32:KERNEL32.dll
 0001:00000040       \177KERNEL32_NULL_THUNK_DATA 0000000180001040     kernel32:KERNEL32.dll
 0001:00000050       MainGuid                   0000000180001050     FileCase.obj
 0001:00000060       MenuGuid                   0000000180001060     FileCase.obj
 0001:00000070       DialogGuid                 0000000180001070     FileCase.obj
 0001:00000080       ??_C@_15NKPPEEJO@?$AA?5?$AA_?$AA?$AA@ 0000000180001080     FileCase.obj
 0001:00000088       ??_C@_13JOFGPIOO@?$AA?4?$AA?$AA@ 0000000180001088     FileCase.obj
 0001:00000090       ??_C@_1DE@BGKMIKPD@?$AAE?$AAu?$AAg?$AAe?$AAn?$AAe?$AA?5?$AAR?$AAo?$AAs?$AAh?$AAa?$AAl?$AA?5?$AA?$CG?$AA?5?$AAF?$AAa?$AAr?$AA?5?$AAG?$AAr?$AAo?$AAu?$AAp?$AA?$AA@ 0000000180001090     FileCase.obj
 0001:000000d0       ??_C@_1FG@IEAGHMHI@?$AAF?$AAi?$AAl?$AAe?$AA?5?$AAn?$AAa?$AAm?$AAe?$AAs?$AA?5?$AAc?$AAa?$AAs?$AAe?$AA?5?$AAc?$AAo?$AAn?$AAv?$AAe?$AAr?$AAs?$AAi?$AAo?$AAn?$AA?5?$AAf?$AAo?$AAr?$AA?5?$AAF@ 00000001800010d0     FileCase.obj
 0001:00000128       ??_C@_1BC@DGHEBOMK@?$AAF?$AAi?$AAl?$AAe?$AAC?$AAa?$AAs?$AAe?$AA?$AA@ 0000000180001128     FileCase.obj
 0001:00000140       ??_C@_1BA@CAKIGJMA@?$AAW?$AAo?$AAr?$AAd?$AAD?$AAi?$AAv?$AA?$AA@ 0000000180001140     FileCase.obj
 0001:00000150       ??_C@_1BG@DFJACJCJ@?$AAP?$AAr?$AAo?$AAc?$AAe?$AAs?$AAs?$AAD?$AAi?$AAr?$AA?$AA@ 0000000180001150     FileCase.obj
 0001:00000168       ??_C@_1BM@BNELJCPP@?$AAP?$AAr?$AAo?$AAc?$AAe?$AAs?$AAs?$AAS?$AAu?$AAb?$AAD?$AAi?$AAr?$AA?$AA@ 0000000180001168     FileCase.obj
 0001:00000188       ??_C@_1BM@HMLICANP@?$AAS?$AAk?$AAi?$AAp?$AAM?$AAi?$AAx?$AAe?$AAd?$AAC?$AAa?$AAs?$AAe?$AA?$AA@ 0000000180001188     FileCase.obj
 0001:000001a8       ??_C@_1BO@IKHLKIJC@?$AAC?$AAo?$AAn?$AAv?$AAe?$AAr?$AAt?$AAM?$AAo?$AAd?$AAe?$AAE?$AAx?$AAt?$AA?$AA@ 00000001800011a8     FileCase.obj
 0001:000001c8       ??_C@_1BI@NPBILFDJ@?$AAC?$AAo?$AAn?$AAv?$AAe?$AAr?$AAt?$AAM?$AAo?$AAd?$AAe?$AA?$AA@ 00000001800011c8     FileCase.obj
 0001:000001e0       ??_7?$DialogItemBinding@UFarDialogItem@@@@6B@ 00000001800011e0     FileCase.obj
 0001:000001f0       ??_7?$DialogBuilderBase@UFarDialogItem@@@@6B@ 00000001800011f0     FileCase.obj
 0001:00000238       ??_7PluginEditFieldBinding@@6B@ 0000000180001238     FileCase.obj
 0001:00000250       ??_7PluginDialogBuilder@@6B@ 0000000180001250     FileCase.obj
 0001:00000298       ??_7PluginCheckBoxBinding@@6B@ 0000000180001298     FileCase.obj
 0001:000002a8       ??_7PluginRadioButtonBinding@@6B@ 00000001800012a8     FileCase.obj
 0001:000002b8       ??_C@_15EFLNJKHH@?$AA?$CF?$AAu?$AA?$AA@ 00000001800012b8     FileCase.obj
 0001:000002c0       ??_7PluginIntEditFieldBinding@@6B@ 00000001800012c0     FileCase.obj
 0001:000002d0       ??_7PluginUIntEditFieldBinding@@6B@ 00000001800012d0     FileCase.obj
 0001:000002e0       ??_C@_11LOCGONAA@?$AA?$AA@ 00000001800012e0     FileCase.obj
 0001:000002e8       ??_C@_1CC@CKMDHNMO@?$AAF?$AAi?$AAl?$AAe?$AAC?$AAa?$AAs?$AAe?$AA_?$AAW?$AAo?$AAr?$AAd?$AAD?$AAi?$AAv?$AA?$AA@ 00000001800012e8     FileCase.obj
 0001:00000310       ??_C@_1BC@ENICKDH@?$AAC?$AAo?$AAn?$AAt?$AAe?$AAn?$AAt?$AAs?$AA?$AA@ 0000000180001310     FileCase.obj
 0001:00000340       __chkstk                   0000000180001340 f   chkstk.obj
 0001:00000340       _alloca_probe              0000000180001340     chkstk.obj
 0001:00000390       ?GetLangString@PluginDialogBuilder@@MEAAPEB_WH@Z 0000000180001390 f i FileCase.obj
 0001:000003a0       ?IsCaseMixed@@YAHPEB_W@Z   00000001800013a0 f   FileCase.obj
 0001:00000430       ?CaseWord@@YAXPEA_WH@Z     0000000180001430 f   FileCase.obj
 0001:00000520       ?DlgProc@@YA_JPEAX_J10@Z   0000000180001520 f   FileCase.obj
 0001:00000560       ?ProcessName@@YAXPEB_WK@Z  0000000180001560 f   FileCase.obj
 0001:00000800       GetGlobalInfoW             0000000180001800 f   FileCase.obj
 0001:00000880       SetStartupInfoW            0000000180001880 f   FileCase.obj
 0001:00000b10       GetPluginInfoW             0000000180001b10 f   FileCase.obj
 0001:00000b60       ?InitDialogItem@?$DialogBuilderBase@UFarDialogItem@@@@MEAAXPEAUFarDialogItem@@PEB_W@Z 0000000180001b60 f i FileCase.obj
 0001:00000b60       ?SaveValue@?$DialogItemBinding@UFarDialogItem@@@@UEAAXPEAUFarDialogItem@@H@Z 0000000180001b60 f i FileCase.obj
 0001:00000b70       ?TextWidth@?$DialogBuilderBase@UFarDialogItem@@@@MEAAHAEBUFarDialogItem@@@Z 0000000180001b70 f i FileCase.obj
 0001:00000b80       ?DoShowDialog@?$DialogBuilderBase@UFarDialogItem@@@@MEAA_JXZ 0000000180001b80 f i FileCase.obj
 0001:00000b90       ??1?$DialogBuilderBase@UFarDialogItem@@@@MEAA@XZ 0000000180001b90 f i FileCase.obj
 0001:00000c10       ?CreateCheckBoxBinding@?$DialogBuilderBase@UFarDialogItem@@@@MEAAPEAU?$DialogItemBinding@UFarDialogItem@@@@PEAHH@Z 0000000180001c10 f i FileCase.obj
 0001:00000c10       ?AddUIntEditField@?$DialogBuilderBase@UFarDialogItem@@@@UEAAPEAUFarDialogItem@@PEAIH@Z 0000000180001c10 f i FileCase.obj
 0001:00000c10       ?AddIntEditField@?$DialogBuilderBase@UFarDialogItem@@@@UEAAPEAUFarDialogItem@@PEAHH@Z 0000000180001c10 f i FileCase.obj
 0001:00000c10       ?GetLangString@?$DialogBuilderBase@UFarDialogItem@@@@MEAAPEB_WH@Z 0000000180001c10 f i FileCase.obj
 0001:00000c10       ?CreateRadioButtonBinding@?$DialogBuilderBase@UFarDialogItem@@@@MEAAPEAU?$DialogItemBinding@UFarDialogItem@@@@PEAH@Z 0000000180001c10 f i FileCase.obj
 0001:00000c20       ??_E?$DialogBuilderBase@UFarDialogItem@@@@MEAAPEAXI@Z 0000000180001c20 f i FileCase.obj
 0001:00000c20       ??_G?$DialogBuilderBase@UFarDialogItem@@@@MEAAPEAXI@Z 0000000180001c20 f i FileCase.obj
 0001:00000c50       ?ReallocDialogItems@?$DialogBuilderBase@UFarDialogItem@@@@IEAAXXZ 0000000180001c50 f i FileCase.obj
 0001:00000d70       ?ItemWidth@?$DialogBuilderBase@UFarDialogItem@@@@IEAA_JAEBUFarDialogItem@@@Z 0000000180001d70 f i FileCase.obj
 0001:00000e00       ?MaxTextWidth@?$DialogBuilderBase@UFarDialogItem@@@@IEAA_JXZ 0000000180001e00 f i FileCase.obj
 0001:00000f20       ?SaveValue@PluginEditFieldBinding@@UEAAXPEAUFarDialogItem@@H@Z 0000000180001f20 f i FileCase.obj
 0001:00000f60       ?InitDialogItem@PluginDialogBuilder@@MEAAXPEAUFarDialogItem@@PEB_W@Z 0000000180001f60 f i FileCase.obj
 0001:00000f90       ?TextWidth@PluginDialogBuilder@@MEAAHAEBUFarDialogItem@@@Z 0000000180001f90 f i FileCase.obj
 0001:00000fa0       ?DoShowDialog@PluginDialogBuilder@@MEAA_JXZ 0000000180001fa0 f i FileCase.obj
 0001:00001040       ?SaveValue@PluginCheckBoxBinding@@UEAAXPEAUFarDialogItem@@H@Z 0000000180002040 f i FileCase.obj
 0001:000010a0       ?SaveValue@PluginRadioButtonBinding@@UEAAXPEAUFarDialogItem@@H@Z 00000001800020a0 f i FileCase.obj
 0001:000010f0       ??0PluginIntEditFieldBinding@@QEAA@AEBUPluginStartupInfo@@PEAPEAXHPEAHH@Z 00000001800020f0 f i FileCase.obj
 0001:000011b0       ?SaveValue@PluginIntEditFieldBinding@@UEAAXPEAUFarDialogItem@@H@Z 00000001800021b0 f i FileCase.obj
 0001:00001200       ??0PluginUIntEditFieldBinding@@QEAA@AEBUPluginStartupInfo@@PEAPEAXHPEAIH@Z 0000000180002200 f i FileCase.obj
 0001:000012c0       ?SaveValue@PluginUIntEditFieldBinding@@UEAAXPEAUFarDialogItem@@H@Z 00000001800022c0 f i FileCase.obj
 0001:00001310       ?CreateCheckBoxBinding@PluginDialogBuilder@@MEAAPEAU?$DialogItemBinding@UFarDialogItem@@@@PEAHH@Z 0000000180002310 f i FileCase.obj
 0001:00001390       ?CreateRadioButtonBinding@PluginDialogBuilder@@MEAAPEAU?$DialogItemBinding@UFarDialogItem@@@@PEAH@Z 0000000180002390 f i FileCase.obj
 0001:00001400       ??_GPluginDialogBuilder@@UEAAPEAXI@Z 0000000180002400 f i FileCase.obj
 0001:00001400       ??_EPluginDialogBuilder@@UEAAPEAXI@Z 0000000180002400 f i FileCase.obj
 0001:00001450       ?AddDialogItem@?$DialogBuilderBase@UFarDialogItem@@@@IEAAPEAUFarDialogItem@@W4FARDIALOGITEMTYPES@@PEB_W@Z 0000000180002450 f i FileCase.obj
 0001:000014e0       ?AddRadioButtons@?$DialogBuilderBase@UFarDialogItem@@@@QEAAXPEAHHQEBH_N@Z 00000001800024e0 f i FileCase.obj
 0001:000016a0       ?AddButtonAfter@?$DialogBuilderBase@UFarDialogItem@@@@QEAAPEAUFarDialogItem@@PEAU2@H@Z 00000001800026a0 f i FileCase.obj
 0001:00001780       ?EndColumns@?$DialogBuilderBase@UFarDialogItem@@@@QEAAXXZ 0000000180002780 f i FileCase.obj
 0001:000018c0       ?UpdateBorderSize@?$DialogBuilderBase@UFarDialogItem@@@@IEAAXXZ 00000001800028c0 f i FileCase.obj
 0001:00001980       ??_GPluginCheckBoxBinding@@UEAAPEAXI@Z 0000000180002980 f i FileCase.obj
 0001:00001980       ??_E?$DialogItemBinding@UFarDialogItem@@@@UEAAPEAXI@Z 0000000180002980 f i FileCase.obj
 0001:00001980       ??_EPluginIntEditFieldBinding@@UEAAPEAXI@Z 0000000180002980 f i FileCase.obj
 0001:00001980       ??_EPluginCheckBoxBinding@@UEAAPEAXI@Z 0000000180002980 f i FileCase.obj
 0001:00001980       ??_GPluginUIntEditFieldBinding@@UEAAPEAXI@Z 0000000180002980 f i FileCase.obj
 0001:00001980       ??_EPluginEditFieldBinding@@UEAAPEAXI@Z 0000000180002980 f i FileCase.obj
 0001:00001980       ??_G?$DialogItemBinding@UFarDialogItem@@@@UEAAPEAXI@Z 0000000180002980 f i FileCase.obj
 0001:00001980       ??_GPluginIntEditFieldBinding@@UEAAPEAXI@Z 0000000180002980 f i FileCase.obj
 0001:00001980       ??_GPluginRadioButtonBinding@@UEAAPEAXI@Z 0000000180002980 f i FileCase.obj
 0001:00001980       ??_EPluginUIntEditFieldBinding@@UEAAPEAXI@Z 0000000180002980 f i FileCase.obj
 0001:00001980       ??_EPluginRadioButtonBinding@@UEAAPEAXI@Z 0000000180002980 f i FileCase.obj
 0001:00001980       ??_GPluginEditFieldBinding@@UEAAPEAXI@Z 0000000180002980 f i FileCase.obj
 0001:000019b0       ?AddIntEditField@PluginDialogBuilder@@UEAAPEAUFarDialogItem@@PEAHH@Z 00000001800029b0 f i FileCase.obj
 0001:00001ac0       ?AddUIntEditField@PluginDialogBuilder@@UEAAPEAUFarDialogItem@@PEAIH@Z 0000000180002ac0 f i FileCase.obj
 0001:00001bd0       ?CaseConvertion@@YAXXZ     0000000180002bd0 f   FileCase.obj
 0001:00002e80       OpenW                      0000000180003e80 f   FileCase.obj
 0001:00002e90       wcsrchr                    0000000180003e90 f   libCRT64:strrchr.obj
 0001:00002ec0       memcpy                     0000000180003ec0 f   libCRT64:memcpy.obj
 0001:00002ef0       ??_V@YAXPEAX@Z             0000000180003ef0 f   libCRT64:delete_array.obj
 0001:00002f00       ??3@YAXPEAX@Z              0000000180003f00 f   libCRT64:delete.obj
 0001:00002f10       ??_U@YAPEAX_K@Z            0000000180003f10 f   libCRT64:new_array.obj
 0001:00002f20       memset                     0000000180003f20 f   libCRT64:memset.obj
 0001:00002f50       ??2@YAPEAX_K@Z             0000000180003f50 f   libCRT64:new.obj
 0001:00002f60       free                       0000000180003f60 f   libCRT64:free.obj
 0001:00002f90       malloc                     0000000180003f90 f   libCRT64:malloc.obj
 0001:00003274       __IMPORT_DESCRIPTOR_KERNEL32 0000000180004274     kernel32:KERNEL32.dll
 0001:00003288       __NULL_IMPORT_DESCRIPTOR   0000000180004288     kernel32:KERNEL32.dll
 0002:00000000       ?ResetButtonID@@3HA        0000000180005000     FileCase.obj
 0002:00000004       ?WordDivEditID@@3HA        0000000180005004     FileCase.obj
 0002:000002a0       ?Opt@@3UOptions@@A         00000001800052a0     FileCase.obj

 entry point at        0000:00000000

 Static symbols

